:020000040801F1
:1000000000000220112401080D120108111201083C
:1000100015120108191201081D1201080000000044
:100020000000000000000000000000002112010894
:100030002512010800000000291201082D120108F4
:100040006124010861240108612401086124010878
:100050006124010861240108612401086124010868
:100060006124010861240108612401086124010858
:100070006124010861240108612401086124010848
:100080006124010861240108612401086124010838
:100090006124010861240108612401086124010828
:1000A0006124010861240108612401086124010818
:1000B0006124010861240108612401086124010808
:1000C00061240108612401086124010861240108F8
:1000D000612401083D120108491201086124010848
:1000E00061240108612401086124010861240108D8
:1000F00061240108612401086124010861240108C8
:1001000061240108612401086124010861240108B7
:1001100055120108612401086124010861240108C5
:100120006124010861240108612401086124010897
:100130006124010861240108612401086124010887
:100140006124010861240108612401086124010877
:100150006124010861240108612401086124010867
:100160006124010861240108612401086124010857
:1001700061240108612401086124010800000000D5
:0801800061240108612401085B
:10018800044B05481B1A062B02D9044B03B1184728
:10019800704700BF4F0000204C0000200000000006
:1001A80005490648091A891001EBD171491002D096
:1001B800034B03B1184770474C0000204C00002047
:1001C8000000000010B5064C237843B9FFF7D8FFAC
:1001D800044B13B10448AFF300800123237010BD12
:1001E8004C000020000000006424010808B5084BFA
:1001F8001BB108490848AFF300800848036813B9E1
:10020800BDE80840CCE7064B002BF9D09847F7E744
:100218000000000050000020642401084C00002069
:100228000000000070B50F4E0F4D761BB61018BFBA
:10023800002405D0013455F8043B9847A642F9D16B
:100248000A4E0B4D761B02F009F9B61018BF0024B0
:1002580006D0013455F8043B9847A642F9D170BD41
:1002680070BD00BF8C2401088C240108902401086B
:100278008C24010870B4860746D0541E002A41D049
:10028800CAB2034602E014F1FF343BD303F8012B52
:100298009D07F8D1032C2ED9CDB245EA05250F2CA0
:1002A80045EA054519D903F110022646103E0F2EDE
:1002B80042F8105C42F80C5C42F8085C42F8045CB6
:1002C80002F11002F2D8A4F1100222F00F0204F099
:1002D8000F041032032C13440DD91E462246043A4B
:1002E800032A46F8045BFAD8221F22F003020432DC
:1002F800134404F003042CB1C9B21C4403F8011BD5
:100308009C42FBD170BC704714460346C2E700BF4D
:1003180081F0004102E000BF83F0004330B54FEAAE
:1003280041044FEA430594EA050F08BF90EA020F1B
:100338001FBF54EA000C55EA020C7FEA645C7FEAAE
:10034800655C00F0E2804FEA5454D4EB5555B8BFD1
:100358006D420CDD2C4480EA020281EA030382EA42
:10036800000083EA010180EA020281EA0303362DD4
:1003780088BF30BD11F0004F4FEA01314FF4801CA7
:100388004CEA113102D0404261EB410113F0004FB9
:100398004FEA03334CEA133302D0524263EB430370
:1003A80094EA050F00F0A780A4F10104D5F1200E0E
:1003B8000DDB02FA0EFC22FA05F2801841F1000169
:1003C80003FA0EF2801843FA05F359410EE0A5F13D
:1003D80020050EF1200E012A03FA0EFC28BF4CF06E
:1003E800020C43FA05F3C01851EBE37101F0004524
:1003F80007D54FF0000EDCF1000C7EEB00006EEB31
:100408000101B1F5801F1BD3B1F5001F0CD34908BA
:100418005FEA30004FEA3C0C04F101044FEA445211
:1004280012F5800F80F09A80BCF1004F08BF5FEA98
:10043800500C50F1000041EB045141EA050130BD78
:100448005FEA4C0C404141EB010111F4801FA4F11B
:100458000104E9D191F0000F04BF01460020B1FA70
:1004680081F308BF2033A3F10B03B3F120020CDAA8
:100478000C3208DD02F1140CC2F10C0201FA0CF086
:1004880021FA02F10CE002F11402D8BFC2F1200CEB
:1004980001FA02F120FA0CFCDCBF41EA0C019040A1
:1004A800E41AA2BF01EB0451294330BD6FEA0404EA
:1004B8001F3C1CDA0C340EDC04F11404C4F12002D5
:1004C80020FA04F001FA02F340EA030021FA04F3E7
:1004D80045EA030130BDC4F10C04C4F1200220FA3E
:1004E80002F001FA04F340EA0300294630BD21FA7C
:1004F80004F0294630BD94F0000F83F4801306BF42
:1005080081F480110134013D4EE77FEA645C18BF35
:100518007FEA655C29D094EA050F08BF90EA020FCC
:1005280005D054EA000C04BF1946104630BD91EAC4
:10053800030F1EBF0021002030BD5FEA545C05D1C7
:100548004000494128BF41F0004130BD14F5800406
:100558003CBF01F5801130BD01F0004545F0FE417A
:1005680041F470014FF0000030BD7FEA645C1ABFAF
:10057800194610467FEA655C1CBF0B46024650EAE6
:10058800013406BF52EA033591EA030F41F4002112
:1005980030BD00BF90F0000F04BF0021704730B598
:1005A8004FF4806404F132044FF000054FF000016D
:1005B80050E700BF90F0000F04BF0021704730B52E
:1005C8004FF4806404F1320410F0004548BF404203
:1005D8004FF000013EE700BF42004FEAE2014FEA58
:1005E80031014FEA02701FBF12F07F4393F07F4F33
:1005F80081F06051704792F0000F14BF93F07F4F65
:10060800704730B54FF4607401F0004521F00041A7
:1006180020E700BF50EA010208BF704730B54FF02D
:1006280000050AE050EA010208BF704730B511F032
:10063800004502D5404261EB41014FF4806404F16A
:1006480032045FEA915C3FF4DCAE4FF003025FEAEC
:10065800DC0C18BF03325FEADC0C18BF033202EB74
:10066800DC02C2F1200300FA03FC20FA02F001FACE
:1006780003FE40EA0E0021FA02F11444C1E600BF6D
:100688004FF0FF3C06E000BF4FF0010C02E000BF56
:100698004FF0010C4DF804CD4FEA410C7FEA6C5C39
:1006A8004FEA430C18BF7FEA6C5C1BD001B050EADC
:1006B800410C0CBF52EA430C91EA030F02BF90EAC7
:1006C800020F0020704710F1000F91EA030F58BF86
:1006D800994208BF90422CBFD8176FEAE37040F0E8
:1006E800010070474FEA410C7FEA6C5C02D150EA86
:1006F800013C07D14FEA430C7FEA6C5CD6D152EA41
:10070800033CD3D05DF8040B704700BF8446104605
:1007180062468C461946634600E000BF01B5FFF704
:10072800B7FF002848BF10F1000F01BD4DF808EDD4
:10073800FFF7F4FF0CBF012000205DF808FB00BFA5
:100748004DF808EDFFF7EAFF34BF012000205DF8FF
:1007580008FB00BF4DF808EDFFF7E0FF94BF01204C
:1007680000205DF808FB00BF4DF808EDFFF7CEFF4D
:1007780094BF012000205DF808FB00BF4DF808ED8C
:10078800FFF7C4FF34BF012000205DF808FB00BF5D
:10079800F0B595B008A830220021FFF76BFD0024C2
:1007A8001D4A019404940394059406940794116CCB
:1007B8001A4B41F080511164126C02F08052019280
:1007C800019A02941A6842F480421A601B680F94D6
:1007D80003F48043029301230225082148220B9346
:1007E80008A803231026109111921393029F0895CD
:1007F8000E9512950C9601F00FF90F224FF48053C5
:1008080003A829460495059407940392069301F0DA
:10081800F9FA15B0F0BD00BF003802400070004082
:1008280010B5214C00F0ECFB01222046114601F0E6
:10083800EDFC20460022022101F0E8FC0A2001F02C
:10084800ADFD20460122022101F0E0FC0A2001F062
:10085800A5FD20460022012101F0D8FC0A2001F064
:100868009DFD20460022022101F0D0FC0A2001F063
:1008780095FD20460122022101F0C8FC0A2001F062
:100888008DFD01221146204601F0C0FC0A2001F02E
:1008980085FD20460022022101F0B8FC0A20BDE8AF
:1008A800104001F07BBD00BF0004024000000000C2
:1008B800674B684A1B88128867496848D1ED007AF7
:1008C80067499FED685A91ED004A07EE103A664B6A
:1008D800F0B5D3ED003A654B05EE902A93ED006A2A
:1008E800634A644BD2ED006AD3ED004A624A634B17
:1008F800B8EEC77A2DED028BE7EE237A83B090ED40
:10090800008AF8EEE55AE7EE246A27EE066AA5EEB5
:10091800848AE7EE067AB0EE667AF3EE096A78EE34
:10092800666AC2ED007AE6EE877A83ED008AF4EE15
:10093800C57AF1EE10FA30DD514B002283ED005AF2
:100948004FF47A746421B5EEC08AF1EE10FA3CD403
:10095800F2EE047A68EE277A4A484B4B0171FDEEB5
:10096800E77A427117EE901AFCEEC87A83FB0132DF
:10097800CB17C3EBA203454E454D316003EB830211
:1009880017EE903AA1EB42020027C27047708370BD
:100998002C6003B0BDEC028BF0BD17EE900AF0EEB0
:1009A800678AFFF719FE28A3D3E90023FFF7C8FEDB
:1009B80090B3334B37491960B5EEC08A0122F1EE86
:1009C80010FA14464FF00001C2D5FAEE047A68EE28
:1009D800277A2C4D2C4B2971FDEEE77AB1EE488A27
:1009E80017EE900AFCEEC87A83FB0031C317274F35
:1009F800274E3860C3EBA10303EB830117EE903A4F
:100A0800A0EB41010120E9706A716870AB70346035
:100A180003B0BDEC028BF0BDF2EE047A68EEA77A63
:100A2800BCEEE87AFDEEE77A0A2317EE904A1448FE
:100A38008DED017A94FBF3F203FB1242D2B29DF8DA
:100A48000410C0ED008A7EE79A9999999999B93F5F
:100A5800AA000020A8000020000000201C000020A0
:100A6800200000200000C8420400002008000020E8
:100A78000C00002010000020A00000206C000020C6
:100A8800A400002014000020676666667800002035
:100A980074000020CDCCCC3D00B587B000230D4AB2
:100AA800009301930393029304930593136B43F00C
:100AB80010031363136B019003F01003009301A953
:100AC80002230548009A039301F084FA07B05DF801
:100AD80004FB00BF003802400004024070B5234EFA
:100AE800234D802400F08CFA348014F003044FF076
:100AF80001021146284604BF2246284601F086FB1B
:100B08000A2001F04BFC01220221284601F07EFB5D
:100B18000A2001F043FC00220221284601F076FB5E
:100B28000A2001F03BFC348864083480002CDCD1B6
:100B38000120FFF7B1FF0A2001F030FC0122022159
:100B48000B4801F063FB0A2001F028FC012108484A
:100B580001F056FB074B224618600221044801F0B9
:100B680055FB0A20BDE8704001F018BC8200002047
:100B7800000402409C00002070B5234E234D8024C1
:100B880000F03EFA348014F005044FF001021146DB
:100B9800284604BF2246284601F038FB0A2001F007
:100BA800FDFB01220221284601F030FB0A2001F05A
:100BB800F5FB00220221284601F028FB0A2001F05B
:100BC800EDFB348864083480002CDCD10120FFF769
:100BD80063FF0A2001F0E2FB012202210B4801F029
:100BE80015FB0A2001F0DAFB0121084801F008FB97
:100BF800074B224618600221044801F007FB0A202F
:100C0800BDE8704001F0CABB820000200004024029
:100C18009C000020F8B5224F224E234D00230120CE
:100C28003B80FFF739FF802333800A2001F0B6FBB1
:100C380001220221284601F0E9FA0A2001F0AEFB60
:100C48000121284601F0DCFA0022022118B13B8874
:100C5800308803433B80284601F0D8FA348864087A
:100C68003480002CE1D100F0CBF9224601210E4856
:100C780001F0CCFA0A2001F091FB012202210A4876
:100C880001F0C4FA0A2001F089FB22460648022135
:100C980001F0BCFA0A20BDE8F84001F07FBB00BFB4
:100CA8008600002082000020000402402DE9F04167
:100CB800264F274E274C284D00233B803380238026
:100CC8002B80FFF7ADFDFFF709FF0120FFF7E4FEDA
:100CD800FA2001F063FB0121204801F091FA18B3D2
:100CE800FFF79EFDFFF748FF0120FFF7D5FEFA202A
:100CF80001F054FB0121194801F082FA60B9184F3C
:100D0800FFF788FF3B882380FFF784FF3B88228812
:100D18002B8043EA02233380FFF7CAFD42F21070AA
:100D2800BDE8F04101F03ABBDFF83480FFF772FF0D
:100D3800B8F800302380FFF76DFFB8F8003022883C
:100D48002B8043EA02233B80CAE700BFA8000020AB
:100D5800AA00002070000020840000200004024047
:100D680086000020484B494A494C80B59A6001F0FA
:100D7800EDFAFFF70DFD00F0A5F800F09DF900F081
:100D880063F900F07DF90A2305224249424800F040
:100D98006FFC4FF47A7001F001FB0A2305223F49EA
:100DA8003D4800F065FC21464FF4FA6314223A48A6
:100DB80000F0BAFC0A2314222146394800F058FCF6
:100DC800A37C5A1E012A57D9052B05D10A230B22C9
:100DD8003449334800F04CFC334C344F344E354DD5
:100DE800B3EE008AFFF762FFD4ED007AF4EEC87A1A
:100DF800F1EE10FAF6D5384600224FF4005101F012
:100E080005FA384600224FF4807101F0FFF93046A8
:100E180000224FF4004101F0F9F9304600224FF466
:100E2800005101F0F3F9304600224FF4006101F05F
:100E3800EDF900224FF400411F4801F0E7F9284678
:100E480000224FF4004101F0E1F9284600224FF456
:100E5800005101F0DBF900224FF40061284601F04F
:100E6800D5F941F2883001F099FA01224FF4005186
:100E7800384601F0CBF9B3E70A2307220F4908489F
:100E880000F0F6FBA8E700BF00ED00E00000010855
:100E9800880000202C0000202C01002024000020C5
:100EA800EC0000203C000020680000200000024008
:100EB800000C0240001002400004024034000020F0
:100EC800704700BF2DE9F0438BB00024464B0094D7
:100ED8001A6B464DDFF82091DFF82081444F454ECC
:100EE80042F001021A631A6B02F001020092009AA2
:100EF80001941A6B42F010021A631A6B02F0100286
:100F08000192019A02941A6B42F002021A631A6B58
:100F180002F002020292029A03941A6B42F008024B
:100F28001A631A6B02F008020392039A04941A6B6C
:100F380042F004021A631B6B03F00403049328466F
:100F480001224FF47841049B01F060F948460122E0
:100F58004FF4404101F05AF9404601224FF47C41D8
:100F680001F054F9384601224FF4007101F04EF9AE
:100F7800012230464FF47C5101F048F9284605A972
:100F880001254FF47843059307940894069501F0DA
:100F980021F8484605A94FF4404305930695079460
:100FA800089401F017F8404605A94FF47C430593CF
:100FB80006950794089401F00DF8384605A94FF4F2
:100FC8000073059306950794089401F003F84FF40D
:100FD8007C5305A93046069507940894059300F0BC
:100FE800F9FF0BB0BDE8F083003802400010024062
:100FF800000802400000024000040240000C0240C9
:1010080030B587B000240E4B00941A6B0D4D42F09A
:1010180002021A631B6B03F00203009328460122A5
:101028000321009B01F0F2F803220123284601A9BD
:10103800039404940192029300F0CCFF07B030BDF2
:1010480000380240000402400B4B0C4A10B50C213A
:101058001A604FF4E134002218465C6059619A60C6
:10106800DA601A619A61DA6100F0D2FA00B910BD4B
:10107800BDE81040FFF724BFEC000020004C004002
:101088000B4B0C4A10B50C211A604FF4E1340022C6
:1010980018465C6059619A60DA601A619A61DA618F
:1010A80000F0B6FA00B910BDBDE81040FFF708BF60
:1010B800AC000020001001400B4B0C4A10B50C216D
:1010C8001A604FF41644002218465C6059619A6011
:1010D800DA601A619A61DA6100F09AFA00B910BD13
:1010E800BDE81040FFF7ECBE2C0100200044004092
:1010F800F0B503683C4A934289B02BD03B4A9342EF
:101108004DD03B4A934201D009B0F0BD0024394B81
:101118000294196C384841F4003119641B6C03F4CB
:10112800003302930322072303A96027022601251F
:10113800DDF808E00692079303970496059500F0FA
:1011480049FF22462146262001F088F8262001F092
:10115800BBF8D9E70024274B0094196C274841F4C1
:10116800002119641B6C03F4002300930322082355
:1011780003A94FF4406702260125DDF800E0069236
:10118800079303970496059500F024FF224621460D
:10119800342001F063F8342001F096F8B4E7002415
:1011A800144B0194596C164841F0100159645B6C5A
:1011B80003F0100301930322072303A9C027022683
:1011C8000125DDF804E00692079303970496059538
:1011D80000F000FF22462146252001F03FF8252097
:1011E80001F072F890E700BF004C00400010014089
:1011F8000044004000380240000C02400008024051
:1012080000040240704700BFFEE700BFFEE700BFD2
:10121800FEE700BFFEE700BF704700BF704700BF92
:10122800704700BF08B501F0ABF8BDE8084001F011
:1012380073B800BF014800F021BB00BFAC0000201C
:10124800014800F01BBB00BF2C010020014800F042
:1012580015BB00BFEC00002008B5032000F0ECFF30
:10126800002211466FF00B0000F0F8FF0022114633
:101278006FF00A0000F0F2FF002211466FF009003B
:1012880000F0ECFF002211466FF0040000F0E6FFCA
:10129800002211466FF0030000F0E0FF0022114623
:1012A8006FF0010000F0DAFF002211464FF0FF3026
:1012B800BDE8084000F0D2BF2DE9F0470468226974
:1012C8008246C068DAF81C10DAF80830DAF81060DC
:1012D800DAF8145022F4405202432261E268DAF844
:1012E8001800334322F416422B4322F00C020B431E
:1012F8001343E360636923F440730343B1F5004F7C
:101308006361AB4B61D09C4200F0018103F58063BF
:101318009C4200F0FC8000F02DFEA64FDAF8043065
:1013280000EB800000EB80009B00B0FBF3F3A7FB11
:1013380003235B091D0100F01DFEDAF8043000EB01
:1013480080009B0000EB8000B0FBF3F600F012FE7B
:10135800DAF8042000EB8000930000EB8000B0FB7B
:10136800F3F3A7FB03234FF064095B0909FB13633D
:101378001B013233A7FB03235B0903F0F00600F0DF
:10138800F9FDDAF8042000EB8000930000EB800000
:10139800B0FBF3F800F0EEFDDAF8043000EB800063
:1013A8009B0000EB8000B0FBF3F0A7FB0030400986
:1013B80009FB10831B013233A7FB0323C3F3431339
:1013C80033432B44A360BDE8F0879C425DD003F50E
:1013D80080639C4259D000F0CDFD764FDAF8043096
:1013E80000EB800000EB80005B00B0FBF3F3A7FB91
:1013F80003235B091E0100F0BDFDDAF8043000EBA1
:1014080080005B0000EB8000B0FBF3F500F0B2FD5C
:10141800DAF8042000EB8000530000EB8000B0FBFA
:10142800F3F3A7FB03235B094FF0640909FB13538C
:10143800DB003233A7FB03231B0903F4F87500F024
:1014480099FDDAF8042000EB800000EB80005300DF
:10145800B0FBF3F800F08EFDDAF8043000EB800002
:1014680000EB80005B00B0FBF3F3A7FB03235B09F1
:1014780009FB1383DB003233A7FB0323C3F34213B7
:1014880033442B44A360BDE8F08700F08BFD494F3F
:10149800DAF8043000EB800000EB80005B00B0FB62
:1014A800F3F3A7FB03235B091E0100F07BFDDAF8C9
:1014B800043000EB80005B0000EB8000B0FBF3F52C
:1014C80000F070FDDAF8042000EB8000530000EB18
:1014D8008000B0FBF3F3A7FB03234FF064095B091B
:1014E80009FB1353DB003233A7FB03231B0903F467
:1014F800F87500F057FDDAF8042000EB800053007F
:1015080000EB8000B0FBF3F800F04CFDA4E700F01E
:1015180049FD284FDAF8043000EB800000EB80002A
:101528009B00B0FBF3F3A7FB03235B091D0100F04D
:1015380039FDDAF8043000EB80009B0000EB8000F6
:10154800B0FBF3F600F02EFDDAF8042000EB800083
:10155800930000EB8000B0FBF3F3A7FB03234FF0ED
:1015680064095B0909FB13631B013233A7FB0323DF
:101578005B0903F0F00600F015FDDAF8042000EB33
:101588008000930000EB8000B0FBF3F800F00AFD48
:10159800DAF8043000EB800000EB80009B00B0FB21
:1015A800F3F3A7FB03235B0909FB138302E700BFDF
:1015B800001001401F85EB512DE9F04107460E460A
:1015C80090461D463C6801E06B1C06D1206836EA4F
:1015D8000003F9D10020BDE8F08135B100F0D8FE54
:1015E800A0EB08008542EDD23C68E36823F4D07391
:1015F800E3606369202223F0010300216361032073
:1016080087F8392087F8381087F83A20BDE8F08144
:1016180060B338B590F83930044603F0FF0203B3DD
:101628002268242384F83930D36823F40053D36024
:101638002046FFF741FE23681A6922F490421A6196
:101648005A6922F02A025A61DA680025202142F4F8
:101658000052DA602846E56384F8391084F83A10B5
:1016680038BD80F83820FFF743FDD9E701207047DF
:101678002DE9F0430F4690F83910202983B003D0A4
:10168800022003B0BDE8F083002F3ED0002A3CD0F2
:10169800984690F83830012B0446F1D000200121FB
:1016A8002123E06384F8381084F83930019200F07F
:1016B8006FFE019AA2848146E28406E0FFF77CFF70
:1016C80028BB23683A785A600137E58CADB24346A7
:1016D8004A4680212046E5B1E58CA668013DADB2B9
:1016E800B6F5805FE584E9D143464A468021204625
:1016F800FFF762FF58B93B8821682269C3F30803E2
:101708004B60002AE0D10237DFE70120B9E7032068
:10171800B7E74021FFF750FF0028F8D1202384F8CD
:10172800380084F83930ACE72DE9F0430E4690F8DC
:101738003A10202983B003D0022003B0BDE8F0831B
:1017480076B36AB3984690F83830012B0446F3D044
:10175800002001212223E06384F8381084F83A300D
:10176800019200F015FE019AA2858146E285E58D79
:10177800ADB243464A462021204685B3E58DA76889
:10178800013DADB2B7F5805FE58512D0FFF714FFD4
:1017980058BB236933B923685B6833700136E6E7C1
:1017A8000120CAE723685B6803F07F0333700136C2
:1017B800DDE743464A4620212046FFF7FDFEA0B953
:1017C800236933B923685B68C3F3080326F8023B2F
:1017D800CDE723685B68DBB226F8013BC7E784F8EE
:1017E8003850284684F83A10A7E70320A5E700BF39
:1017F800704700BF704700BF8368B3F5805F28D08B
:10180800036973B10368826A5B68511C03F07F0344
:1018180081621370C38D013B9BB2C38543B1002025
:101828007047836A0268591C526881621A70F1E72E
:101838000268D16821F4907110B5D16051692024F3
:1018480021F00101516180F83A40FFF7D3FF0020F1
:1018580010BD0269836A3AB902685268C2F3080285
:1018680023F8022B8362D5E702685268D2B223F8C4
:10187800012B8362CEE700BF704700BF03681A6878
:1018880070B51607DD685969044649D011F00101A1
:1018980052D0D60705D5E80503D5E06B40F0010026
:1018A800E06356077AD5002900F08480E16B900741
:1018B80041F00201E16376D5E16B41F00401E16397
:1018C800110772D4E16B002929D0910605D5AA0623
:1018D80003D594F83A20222A7CD05D69E16B0E0783
:1018E80002D415F040057AD0DA6822F49072DA60F2
:1018F8005A69202122F001025A6184F83A105A6983
:1019080055065ED55A69606B22F040025A6100287C
:1019180057D03B4B036500F07DFC002855D170BDC6
:1019280096060CD5A9060AD590F83A30222BF6D19E
:10193800BDE87040FFF760BF15F4907FA9D110068D
:101948000ED45606EBD56D06E9D5DA68202122F0CB
:101958004002DA60204684F83910FFF749FF70BD6D
:101968002906EED594F83920212AD8D1A268B2F5F3
:10197800805F226A38D0511C216212785A60E28C4A
:10198800013A92B2E284002AC9D1DA6822F08002D0
:10199800DA60DA6842F04002DA6070BD96070BD56B
:1019A800002989D18EE711078CD5E16B41F0080138
:1019B800E16387E7900785D4100783D5002981D094
:1019C800F3E72046FFF758FF70BD606BBDE8704035
:1019D800036D18472046FFF70FFF23687DE7204671
:1019E800FFF74AFFE56370BD11882069C1F308015C
:1019F800596010B902322262C1E701322262BEE7A1
:101A08000D1A010808B5836B0022DA851846DA84B6
:101A1800FFF732FF08BD00BFF0B50368DD0783B0EC
:101A280004462FD5A3498A6802F00C02042A00F064
:101A3800F4808A6802F00C02082A00F0EA806368E1
:101A4800B3F5803F00F02C81B3F5A02F00F00081A2
:101A5800984D2A6822F480322A602A6822F480226B
:101A68002A60002B40F0FD8000F092FC064605E05D
:101A780000F08EFC801B642800F2AA802B689B0370
:101A8800F6D423689F072DD58A4A916811F00C0F68
:101A980000F0A580916801F00C01082900F09B80F6
:101AA800E368002B00F0EB80834B824D01221A6023
:101AB80000F06EFC064605E000F06AFC801B022878
:101AC80000F286802B689807F6D52968F82292FAE2
:101AD800A2F22369B2FA82F221F0F80193400B4393
:101AE8002B6023681A0720D4590734D4A369CBB1D3
:101AF800704DAA6802F00C02082A77D0022B6F4BAF
:101B08004FF000021A6000F0D18000F041FC2C4632
:101B1800054604E000F03CFC401B022858D8236826
:101B28009B01F7D4002003B0F0BD6369002B60D09F
:101B3800634B604D01221A6000F02AFC064604E05F
:101B480000F026FC801B022842D86B6F9F07F7D550
:101B580023685907CAD5574B5A4D002201921A6C6F
:101B680042F080521A641B6C03F080530193019B6E
:101B78002B6843F480732B6000F00AFC064604E0EF
:101B880000F006FC801B022822D82B68DA05F7D55E
:101B9800A368012B00F0F180052B00F0D580454D9E
:101BA8002A6F22F001022A672A6F22F004022A67AC
:101BB800002B40F0D28000F0EBFB41F2883607465C
:101BC8002B6F980792D500F0E3FBC01BB042F7D902
:101BD800032003B0F0BD526856023FF561AF354AA5
:101BE8001268950723D5E268012A20D0012003B0A6
:101BF800F0BD334A2F4D136000F0CAFB064604E0DF
:101C080000F0C6FB801B0228E2D86B6F9807F7D458
:101C18009EE74A6850027FF512AF264A1268910380
:101C28007FF530AF6268002A7FF42CAFDEE7214DE4
:101C3800F821286891FAA1F12269B1FA81F120F01E
:101C4800F8008A4002432A601A077FF54DAF6CE717
:101C5800184B1A6842F480221A601A6842F48032DB
:101C68001A6000F095FB134D064604E000F090FB67
:101C7800801B6428ACD82B689A03F7D501E70E4A75
:101C88000C4D136000F084FB064604E000F080FB76
:101C9800801B02289CD82B689907F7D4236821E772
:101CA800044A136843F480331360DAE700F070FBEA
:101CB80006460FE0003802400000474260004742F5
:101CC800800E47420070004000F062FB801B022833
:101CD8003FF67EAF2B689901F6D447F6C07696FAA0
:101CE800A6F64FF44032B6FA86F692FAA2F24FF010
:101CF8007061B2FA82F091FAA1F1A26A676AE369A7
:101D0800D4F820E0E46A520843EA0E0307FA06F61C
:101D1800013A8240B1FA81F1334304FA01F11343E5
:101D2800194A1A4C0B4301216B60116000F030FB1B
:101D3800054605E000F02CFB401B02283FF648AFA3
:101D480023689A01F6D5EDE6104B1A6F42F00402AB
:101D58001A671A6F42F001021A6700F019FB0B4D5F
:101D6800074641F288362B6F9B073FF5BFAE00F060
:101D78000FFBC01BB042F6D92AE7044A136F43F0A1
:101D880001031367E9E700BF6000474200380240DB
:101D9800194A936803F00C03042B2BD0082B27D186
:101DA8005168536801F03F0113F4800F536847F6F8
:101DB800C07292FAA2F0B0FA80F003EA020323FAA2
:101DC80000F314BF0D480E48B0FBF1F000FB03F020
:101DD800094B4FF440325B6892FAA2F2B2FA82F2EF
:101DE80003F44033D34001335B00B0FBF3F070479A
:101DF80003487047014870470038024040787D0129
:101E08000024F400574A136803F00F038B4208D2EA
:101E1800CBB21370136803F00F03994201D001206D
:101E2800704703689A072DE9F04106D54E4C85683E
:101E3800A26822F0F0022A43A260DF0706460C4699
:101E480026D54268012A00F08780931E012B464B55
:101E58001B687BD9990728D5434DAB6823F003034A
:101E68001343AB6000F094FA7368012B074641F204
:101E780088384FD0022B58D0032B05D160E000F0F2
:101E880087FAC01B404564D8AB6813F00C0FF6D135
:101E9800344A136803F00F039C4209D2E3B213706B
:101EA800136803F00F039C4202D00120BDE8F081C3
:101EB80033685A0706D52C49F0688A6822F4E0523C
:101EC80002438A601B0707D5274A3169936823F4C0
:101ED800604343EAC1039360FFF75AFF224B014670
:101EE800F0229B6892FAA2F2B2FA82F203F0F003AF
:101EF800D3401E481E4AC35C002021FA03F3136036
:101F080000F00EFA0020BDE8F08100F041FAC01B95
:101F180040451ED8AB6803F00C03042BF5D1B7E796
:101F280000F036FAC01B404513D8AB6803F00C0329
:101F3800082BF5D1ACE700F02BFAC01B404508D8B8
:101F4800AB6803F00C030C2BF5D1A1E7980183D4FF
:101F5800ABE70320BDE8F081034B1B689D033FF509
:101F68007BAFA2E7003C0240003802407C24010815
:101F780048000020084B4FF4E0529B6892FAA2F206
:101F8800B2FA82F203F4E053D3400449044ACB5C2A
:101F98001068D840704700BF003802407C24010810
:101FA80048000020084B4FF460429B6892FAA2F266
:101FB800B2FA82F203F46043D3400449044ACB5C8A
:101FC8001068D840704700BF003802407C240108E0
:101FD800480000202DE9F04FD1F800C0DFF8148246
:101FE800DFF814E283B0002503E00135102D00F07E
:101FF8009B800123AB4003EA0C029342F5D14E6863
:1020080026F0100ABAF1020F00F091804FEA450954
:102018000324D0F800B004FA09F4E44306F00307F7
:102028000BEA040B07FA09F70AF1FF3A47EA0B072C
:10203800BAF1010F076040F2A080C7688B683C4086
:1020480003FA09F32343C360F300CED54FF0000928
:10205800CDF80490D8F8443043F48043C8F84430AD
:10206800D8F8444025F0030303F1804304F4804486
:1020780003F59C33019405F00304019FD3F808A0ED
:10208800A4000F27A7402AEA070A544FB84222D0D3
:1020980007F58067B84200F08380514FB84200F0DE
:1020A8008480504FB84200F085804F4FB84200F00E
:1020B80086804E4FB84200F087804D4FB84200F0FE
:1020C8008880DFF8389148450CBF4FF007094FF07A
:1020D800080909FA04F94AEA09079F60DEF800309E
:1020E800D443F70354BF23401343CEF80030DEF83F
:1020F8000430B70354BF23401343CEF80430DEF84E
:102108000830F70254BF23401343CEF80830DEF8F6
:102118000C30B60205F1010554BF23401343102DBE
:10212800CEF80C307FF465AF03B0BDE8F08F4FEA0E
:10213800D50900EB890905F00707D9F82040BF0049
:102148004FF00F0B0BFA07FB24EA0B0A0C69BC4093
:1021580044EA0A04C9F820404FEA45090324D0F8A4
:1021680000A004FA09F4E44306F003070AEA040AA3
:1021780007FA09F747EA0A070760876807EA040ABF
:10218800CF6807FA09F747EA0A078760D0F804A07A
:10219800C6F300172AEA0303AF401F4347604CE722
:1021A8004FF0010909FA04F995E74FF0020909FA15
:1021B80004F990E74FF0030909FA04F98BE74FF0A7
:1021C800040909FA04F986E74FF0050909FA04F940
:1021D80081E74FF0060909FA04F97CE7000002409C
:1021E80000080240000C02400010024000140240A7
:1021F8000018024000380240003C0140001C024028
:102208000369194214BF01200020704702B909046C
:102218008161704790F83530022B03D080234365E5
:10222800012070470268052380F83530136823F0D1
:102238000103136000207047074AD3684FF6FF0177
:102248000B40000243F0BF6300F4E06043F4003346
:102258000343D360704700BF00ED00E0184B70B433
:10226800DC68C4F30224C4F10706042E04F1040355
:1022780028BF0426062B17D9033C0125A540013D9C
:102288002A400123B340013B1940A140002841EAFC
:1022980002010CDB00F1604000F561400901C9B2A0
:1022A80080F8001370BC704700221446E9E7054B1C
:1022B80000F00F0009010344C9B2197670BC7047D9
:1022C80000ED00E0FCEC00E000F01F0101234009F4
:1022D800024A8B4042F82030704700BF00E100E01E
:1022E8000138B0F1807F0ED2084B10B4084C58600A
:1022F800F02084F823000022072110469A60196014
:102308005DF8044B70470120704700BF10E000E003
:1023180000ED00E0704700BF08B5FFF7FBFF08BD00
:10232800084B094A1B6810B5A2FB03230446980909
:10233800FFF7D6FF214600224FF0FF30FFF78EFF50
:10234800002010BD48000020D34D621008B50B4B8B
:102358001A6842F400721A601A6842F480621A60BD
:102368001A6842F480721A600320FFF765FF0020A4
:10237800FFF7D6FFFEF770FF002008BD003C0240C3
:10238800024A136801331360704700BF6C010020D4
:10239800014B1868704700BF6C01002010B582B06F
:1023A8000190FFF7F5FF0446FFF7F2FF019B001BC2
:1023B8009842F9D302B010BD1049114BD1F88820CA
:1023C80042F4700210B4C1F888201A680D4C00203D
:1023D80042F001021A6098601A6822F0847222F4AE
:1023E80080321A605C601A684FF0006422F4802220
:1023F8001A60D8608C605DF8044B704700ED00E00F
:102408000038024010300024DFF834D0002103E007
:102418000C4B5B58435004310B480C4B42189A4202
:10242800F6D30B4A02E0002342F8043B094B9A42D8
:10243800F9D3FFF7C1FFFDF7F5FEFEF793FC7047F0
:102448000000022094240108000000204C00002015
:102458004C00002070010020FEE70000F8B500BF26
:10246800F8BC08BC9E467047F8B500BFF8BC08BC6D
:042478009E467047C5
:10247C00000000000102030401020304060708091E
:04248C00F50101084D
:04249000CD01010871
:10249400C5FE02C0BD52163DF624D6B50AD7233C6C
:1024A400ACC5A738FF00000000000D0066661EC220
:1024B4000AD7233CFE00010001000000FE000200D8
:1024C40002000000636F6E6E656374006E6F7420AB
:0C24D400636F6E6E656374000024F400FA
:0400000508012411B9
:00000001FF
